:020000020000FC
:0400000009C053C020
:0200080083C0B3
:10000C006DC078C082C039C10FEF07BB0FEF08BBC2
:10001C0008E004BB07E305BB0BE101BB00EE02BB30
:10002C000FE50DBF04E00EBF51E033247724882781
:10003C009927AA27CC27DD276627772703E0602E90
:10004C000FEF802E0FEBC02ED02EE02EF02E0027BF
:10005C0000936000009361000FEF00936200009327
:10006C0063000EEF402E502E04E003BF00E00FBDE6
:10007C0003E00EBD00E00BBD00E10ABD00E009BDD0
:10008C0000E408BD04E005BD0DE509BF01E805BFAE
:10009C0000E40BBF00E808B978948895FECF000007
:1000AC00B0B3B470B81509F418958B2EB2FF07C015
:1000BC008CB59DB58031970580F074BC189584B5CE
:1000CC00883058F07DBC7CBC803830F0AA24BB242E
:1000DC0099243324AA2701C0A82F1895A83048F0DA
:1000EC00B2FD07C0AA0CBB1C991C3394A03208F0BB
:1000FC00A3941895B2FD05C00CD0AA24BB24992456
:10010C003324189501E804BD18950FEF7DBC0CBD88
:10011C00189508E1301609F401D008959501492D80
:10012C0013B31470032F08700695101709F0089577
:10013C008901102702951027012F16951695012776
:10014C00102F169501270170132F1295117010178F
:10015C0009F00895032F142F009510951695079507
:10016C001695079516950795169507951695079567
:10017C0037700217130709F008952901B90104D04B
:10018C00AB9AC0E7D7E1089510916300009162002B
:10019C006017710720F470936300609362001091F4
:1001AC006100009160000617170720F4709361003E
:1001BC006093600060FC04C0709163006091620009
:1001CC0061FC04C070916100609160007E3F09F495
:1001DC004EC06F3F07E0700708F043C0613000E08D
:1001EC00700708F438C0CC24DD24EE24FF2411E081
:1001FC00643F710718F0645F714007C004EF11E0B1
:10020C00061B170BB8010AE0F02E683E03E07007DE
:10021C0020F0685E7340F394F8CF643600E070070A
:10022C0020F064567040E394F8CF6A3018F06A50AE
:10023C00D394FBCF062F67D0C02E0D2D64D0D02EBB
:10024C000E2D61D0E02E0F2D003011F05CD001C0CE
:10025C000FEFF02E089507EFC02ED02EE02EF02ECB
:10026C0008950EEFC02ED02EE02EF02E08950FEB39
:10027C00C02ED02EE02EF02E089502EB02BF5A9520
:10028C0009F454E001D0189500EE02BBE0E5F1E072
:10029C00E50FF71D09940FC00AC004C000C0C8BA0E
:1002AC00909A08950D2D0F7708BB919A0895E8BA8E
:1002BC00939A0AD00895F8BA949A01D00895C1502F
:1002CC00D04009F4AB980895112703B303700611BD
:1002DC001FEF602E003039F01F3F21F4033009F47A
:1002EC00B20168DF0895002700936000009361005D
:1002FC000FEF00936200009363000FEBC02ED02E23
:10030C00E02EF02E08950B3008F00BE0F3E0E4E261
:10031C00E00FF71D04910895C0F9A4B0999282F8EA
:04032C008090BF8678
:00000001FF
